:020000040800F2
:1000000000200020692F0008E9200008EB200008EC
:1000100000000000000000000000000000000000E0
:10002000000000000000000000000000ED200008BB
:100030000000000000000000EF20000865430008F9
:10004000E92F0008E92F0008E92F0008E92F000830
:10005000E92F0008E92F0008E92F0008E92F000820
:10006000E92F0008E92F0008E92F0008E92F000810
:1000700081430008E92F0008E92F0008A9140008AF
:10008000E92F0008E92F000800000000E92F000810
:10009000E92F0008E92F0008E92F0008FD110008EA
:1000A000E92F0008E92F0008E92F0008E92F0008D0
:1000B0002143000800000000E92F000800000000B4
:0400C0005FF808F1EC
:1000C80002B4714649084900095C49008E4402BCE3
:1000D8007047C046002934D00123002210B488425A
:1000E8002CD301242407A14204D2814202D209015F
:1000F8001B01F8E7E400A14204D2814202D2490080
:100108005B00F8E7884201D3401A1A434C08A04222
:1001180002D3001B5C0822438C08A04202D3001BB8
:100128009C082243CC08A04202D3001BDC082243CF
:10013800002803D01B0901D00909E3E7101C10BCF3
:100148007047002801D00020C04307B4024802A12C
:100158004018029003BDC046190000000029F0D0E5
:1001680003B5FFF7B9FF0EBC4243891A1847C046CA
:100178007047C0460020704770470020704770479E
:1001880000207047034A002312684370826183701D
:100198007047C0460000002043788B4205D0034BCF
:1001A80000221A8101230170837070470403002024
:1001B80003681B021B0E01D102238370704703687A
:1001C8001B021B0E01D1032383707047124B70B5BD
:1001D8005E890F21B6B23140051C043000F09AFC4C
:1001E8000E4CF606231C38331B78F60FB3420ED09C
:1001F800002B01D00A4B00E00A4BE069236002F0B3
:100208006DF8E069211C383402F082F82670A8697C
:100218000368DB68984770BD04030020840300204E
:1002280023097200220C941070B58069064C03688B
:10023800251C54352E889B6898472B88B6B29E4259
:1002480001D15034208070BD04030020F8B5041C8F
:1002580000680002000E04286CD8FFF731FF031E67
:10026800474E5200201CFFF7DFFF334D201C2B1C8C
:10027800503319880C3009B200F058FC63892269A0
:100288005235D31A62681BB29B18227A63601341F5
:1002980063819B049B0C2B804CE0A06903685B681E
:1002A80098472378244D092B1AD8244E9A00905940
:1002B800037103681B689847071E0FD12378201C19
:1002C8009B009B59A361FFF781FFA06903681B6925
:1002D8009847A88158352F8004232AE03668A661FC
:1002E80054352B8801339BB22B8021E0A069036829
:1002F8001B699847104B98811AE0201CFFF766FF8E
:1003080016E0201CFFF790FF0B4B1A1C583212887E
:10031800002A0FD02278012162701A8150331B887D
:1003280021751AB2A3816381237A22619A4062609F
:100338000023A370F8BDC04604030020000000207D
:100348000A4A0B4B0B481A600B4B0C4A0C491861B4
:1003580058610C485A60DA601A625A62996098616A
:10036800D961094A094B1A607047C046F031000844
:1003780048000020C003002000000020DC0300200B
:10038800FC020020AC020020500000206C0000207D
:10039800044B20211A8801321A80034B1A880A4319
:1003A8001A8070477000002072000020031CFF3381
:1003B8009A790379D01A80B27047021C0379FF3208
:1003C80091795A1C0271994202D9C018807900E0CB
:1003D8000020704710B5021CFF329379FF2B03D021
:1003E8005C1CC3189471997110BD10B5031CFF33C0
:1003F80099790022031C1C1AE4B28C4204D29C791D
:1004080001331219D2B2F6E7101C10BD08B5044822
:10041800044900220C2301F0B1FC00F039FA08BDB0
:10042800740000202032000800B50B4BC3B00093C5
:100438006A46432353710023FF32011C93716846B7
:100448006A461371FFF7C6FF044B6946186800F047
:10045800EDF943B000BDC04610320008C0020020CC
:10046800024B034A1A60034A5A607047740000201E
:10047800004300080044004008B50520404202F04F
:10048800A1F9054802F0ACF9012002F0C3F90120F6
:1004980002F0ACF908BDC046808D5B00094B012213
:1004A80030B51A601C68084A084954438D68641BB3
:1004B8000625684320181C688D685443641B8442D1
:1004C800F9D330BDA0020020808D5B0010E000E071
:1004D800094B012230B51A601C68084A0849544380
:1004E8008D68641B074D684320181C688D68544349
:1004F800641B8442F9D330BDA0020020808D5B00CC
:1005080010E000E0701700007047704770477047B0
:10051800704770470B4A0C4B5089191DC8871089C2
:10052800991DC887D088191C0831C8879088191C5C
:10053800483108805088191C4A31088012884C3389
:100548001A807047ACF7FF1F0403002008B50B485A
:1005580002F0F2FB01F094FF094B0020186058608C
:10056800986001F0BDFF012383F31088054B1B68D9
:1005780083F30888044B1B68984708BD003801407E
:1005880010E000E000ECFF1F04ECFF1F08B5012895
:1005980002D101F049FCFEE7FFF7D8FF08BD0020B3
:1005A80070477047F0B5071C80208BB0800201218E
:1005B80002F070F880208000012102F077F8902086
:1005C800032302A900250126C0050B7104ACCD71D7
:1005D800029601F011FE1C4801F09AFD201C01F062
:1005E800BFFD1948211C04952671A5602561656128
:1005F80001F0A0FD311C1448072201F0C1FD12488A
:1006080001F0C3FD1048311C01F0B2FD0E48012174
:1006180001F0E2FD0028F9D001A80C2303700124A1
:1006280003234370847001F0FBFE221C0421002484
:10063800054801F0C8FDBC60BC81034801F0BBFD62
:10064800201C0BB0F0BDC0460024014007B50021B6
:10065800094801F08DFD684601F00CFE9020012349
:10066800C0056946009301F0C7FD0348034901F03E
:10067800B3FD0128F9D007BD0024014001000001A5
:1006880070B58189041C0F4D002913D00E4B8026AC
:100698007601DE67836858359800FFF71BFD2B88C5
:1006A80080B201339BB22B800023A360A381074B48
:1006B8001E6005E054352B88081C01339BB22B8043
:1006C80070BDC0460403002004E100E000E100E042
:1006D800024A034B08321A607047C046603200086D
:1006E800AC02002038B50368041C5B68984723688F
:1006F800051C5B68201C98470002281800B238BD0A
:1007080038B50368041C0D1C9B68C9B29847236858
:100718002D12E9B29B68201C984738BDF8B5041C17
:1007280000680D1C0368DB689847002871D026799B
:10073800012E15D0002E02D0022E33D069E0206899
:1007480003685B689847031C20683E2B04D1036844
:100758001B68984701235FE003685B69984758E086
:1007680020680368DB689847022852D92068036824
:100778001B6898472072206803681B689847E080C8
:10078800A568636820681B0CEDB2ED180368EDB22C
:100798001B689847854241D163681B0CFF2B3DD8E5
:1007A800022339E0206866680368360CDB689847DE
:1007B80086422EDAA3682E1C6B71FF360023B371B4
:1007C8002B716268B179120C2B68914208D22068AB
:1007D8009F6803681B689847011C281CB847F0E706
:1007E8000026281C2671DB689847051C20680268CB
:1007F8001268904785420AD10B4B20681A8820213D
:100808008A431A8003689B699847012002E0FFF732
:10081800BFFD002040B2F8BD2371FAE7FFF7B8FD2D
:1008280000202071F6E7C04672000020F8B5046881
:100838000D1C2368201C9B683E2198472368697912
:100848009B68201C98472F1C2368FF37B9799B6841
:10085800201C9847B9796A7923688918C9B29B68B6
:10086800201C98470026BA792368B24207D9AA19EA
:1008780091799B68201C01369847F6B2F3E79E6889
:100888002B68281CDB689847011C201CB047F8BD62
:10089800044B054A05491A6000221A710A70044A75
:1008A80013607047C802002074000020C4020020B2
:1008B800C002002030B5041C407985B042380023BE
:1008C800142800D9DAE0FFF7FBFB9B7DD94BD975DB
:1008D800D9D9D9D9D9B1C9D932D9D9D9D98A0B0055
:1008E800221CFF32937123712368201C9B685521B9
:1008F8009847201C7921FFF703FF2368201C9B6879
:1009080000219847201CAA21FFF7FAFE2368201C23
:100918009B68FF2198470C25013DEDB2002D00D1C1
:100928009AE02368201C9B6800219847F4E7201C64
:10093800FFF7D8FE051C201CFFF7D4FE231CFF334D
:100948009A79237900249A4200D098E04D4B81B2DD
:10095800AAB2186800F01EFE5020FFF765FD8EE071
:100968002368201C5B689847464B041E10D0186803
:1009780001240470002100F057FE211C424802F0B7
:1009880061F89020C0050421221C01F08FFC0FE0C3
:100998001D689020C0050421221C01F087FC281C3A
:1009A800211C00F041FE2C703748211C02F04AF847
:1009B800452011E0221CFF3293712371334B5233CF
:1009C800198845E02368201C5B689847304B011C58
:1009D8001868FFF7E1FB4320FFF726FD4EE0221CD5
:1009E800FF32937100252371284A2368AA184232DE
:1009F80011789B68201C01359847062DF4D12BE00F
:100A08002368201C5B6898476D460E350223021C3C
:100A1800009331212B1C1F4800F042F9221C0023AF
:100A2800FF32937123710023E95E12E02368201CD2
:100A38005B689847221C0023FF32937123713F287B
:100A480002D9154B198802E0104B4000C15A89B2EF
:100A580009B2201CFFF754FE012410E0221CFF32CB
:100A6800937100252371094B6A00D15A201C09B2E1
:100A78000135FFF745FE402DF5D1EDE70024201C98
:100A880005B030BDD0030020002C01400403002035
:100A98006C000020F40200204400002030B5174B01
:100AA800C3B0174D009300232B702978154C164BB3
:100AB80000291AD123601B68002B13D01348032286
:100AC80002F02EFB20686946FFF728FE002809D0AF
:100AD8006846FFF7EFFE0028F4D020686946FFF764
:100AE800A5FEEFE72B780133DEE7094A0C211278DF
:100AF8004A439B18236043B030BDC04610320008FB
:100B0800BC020020C0020020C8020020D40200203D
:100B1800C402002003790268994202D9CB1A9A408C
:100B280001E05B1A1A41026001717047037A10B53F
:100B3800002B17D0028880248A1A92B293B20180BF
:100B480019B2A401A14201DD094904E0094CA142FE
:100B580003DA8021C90153189BB242681BB2D3182B
:100B6800436003E0012301804160037210BDC04669
:100B780000C0FFFF00E0FFFFF7B5051C8020C002A2
:100B8800012101F087FD6A4602231E4F13710323DA
:100B98005371802300240126381CDB0069469671B6
:100BA800D471009301F028FB80231B01381C69468F
:100BB800009301F021FB381C321C0A2101F07CFB58
:100BC800321C381C0B2101F077FB8020311CC0033C
:100BD80001F078FD286801F081FB0B490B4A286871
:100BE8000A60CC604C608C600C614C618C6101F0D7
:100BF8008FFB2868311C01F0BDFB286801F0C4FB9D
:100C0800AC80F7BD00040048D8020020220C9410E4
:100C180038B5064D064C074B281C236001F05EFBD7
:100C2800281C211C01F074FB38BDC0460058004048
:100C3800D80200202309720038B5064D064C074B30
:100C4800281C236001F04AFB281C211C01F060FBD2
:100C580038BDC04600580040D8020020220C94102D
:100C6800F8B50D4E0D4B041C0F1C33602068391C61
:100C780001F0ABFB00280CD135686B1E3360002DEA
:100C8800F4D1A38820680133A38001F07DFB281CE0
:100C980000E00120F8BDC0462C000020102700000D
:100CA800F0B587B0049383884E00059380239B0199
:100CB8000093041C311C0068151C002301220C9FA2
:100CC80001F06CFB201C0221FFF7CAFF002801D1AC
:100CD8000020A4E02068291C01F072FB201C4021A0
:100CE800FFF7BEFF0028F3D0FF21381CFFF7F2F909
:100CF800FF210390381CFFF731FA039B0D1C002BD2
:100D080072D00127039B2068012B10D1002D0ED132
:100D1800002F03D090239B01009300E000958023CF
:100D2800311CFF229B0401F039FB002713E0002F40
:100D380003D090239B01009300E000978023311C8F
:100D4800FF225B04EFE7206801F03CFB049BD855C9
:100D58000137FF2F06D0201C0421FFF781FF002850
:100D6800F1D1B5E7FF330493039B013B0393002BB9
:100D780007D0201C80210027FFF772FFB842C1D19D
:100D8800A6E7002D10D1201C2021FFF769FF0028BD
:100D98009ED02068202101F01EFB059BA088C01A68
:100DA80043425841C0B23AE0201C8021FFF758FF67
:100DB80000288DD0039BEAB200938023311C206861
:100DC8009B0401F0EBFA049E7519201C0421FFF71F
:100DD80047FF002800D17BE7206801F0F3FA307064
:100DE8000136AE42F1D1CEE790239B0100938023D8
:100DF800CAB22068311C9B0401F0D0FA049E751910
:100E0800AE42C0D0201C0421FFF72AFF002800D1E1
:100E18005EE7206801F0D6FA30700136F0E707B0D7
:100E2800F0BD704770470000F0B5037985B0061C27
:100E38001D4D4179022B0FD1012402AB0094281CCF
:100E4800FC22FFF72DFF6B467179281C0094FB22CA
:100E58000933FFF725FF1EE003AC022300931B2292
:100E6800231C281CFFF71CFF6278237812111B0132
:100E7800D318717902AF01263B700B220096231C10
:100E8800281CFFF70DFF23781A1116400822B60018
:100E98001340F3187B7002AB58781B7800021818BF
:100EA80080B205B0F0BDC046F40200207FB5304CDA
:100EB800051C201CFFF760FE201CFFF7BDFE206804
:100EC80001F062FA2B79022B2AD140236B71052697
:100ED800012300936979201CFC2203ABFFF7E0FE95
:100EE800002801D101203FE0013EF6B2002EEFD1EB
:100EF800201CFFF78DFE0526012300936979201C2D
:100F0800FC2203ABFFF7CCFE002803D1201CFFF71F
:100F180093FE03E0013EF6B2002EEDD1002023E05F
:100F280036236B710526012300936979201C1B2247
:100F380003ABFFF7B5FE0028D4D0013EF6B2002E71
:100F4800F1D1201CFFF764FE05260123009369797F
:100F5800201C1B2203ABFFF7A3FE0028D6D0013EBE
:100F6800F6B2002EF1D1D9E70023A38004B070BDFA
:100F7800F402002030B50379021C85B01948517974
:100F880003AC194D022B10D10093FE22231CFFF74E
:100F980087FE00281ED058352B88207801339BB255
:100FA8002B806378800118181AE0022300930C2222
:100FB800231CFFF775FE00280CD058352B882078A5
:100FC80001339BB22B800F23184063780002181856
:100FD800800005E054352B88002001339BB22B801C
:100FE80005B030BDF402002004030020034B044A7E
:100FF8001A60044A044B08321A607047F402002051
:101008000058004080320008FC020020C3697621A5
:101018001A6810B58A431A6099690122090C1140AF
:10102800841CE177002907D18022520042841A6883
:101038007C210A431A6009E0448C411DCC77196869
:101048007A242143196099690A439A612E300278FB
:1010580001218A4302700822DA6110BDC369064A79
:1010680059680A405A601A6876218A431A601A68D1
:1010780088210A431A607047FF7FFFFFF8B5C369EC
:101088001022996911420DD19A69110702D5FFF70B
:10109800BDFF2CE099692022114203D19A69940777
:1010A80004D424E0DA61FFF7D9FF20E0021C2E32D5
:1010B8001478E407E40FE4B2002C0BD1451DE97F56
:1010C800866A4F1CEF77FF253F2902D849008D5BC0
:1010D800ADB285850019283001799962137801210C
:1010E800D807C00F0C1C84438B4323431370F8BDEF
:1010F80038B5C369FA229969041C114204D01968E9
:101108007A220A407A2A09D09969FC22114208D029
:1011180019687C220A407C2A03D10AE0FFF7AEFF57
:1011280066E099690822114262D01B68134209D10E
:101138005EE099691022114201D0DA6158E09A699B
:10114800110703D5201CFFF761FF51E09A69510789
:1011580004D49969202211422AD149E0618C802265
:101168005200914204D15B6A63840534E3773FE01F
:10117800221C2E321178586AC907C90FC9B26318E0
:1011880028331871012909D1611DCB7FA06A5D1C24
:10119800CD77A18D1F2B01D85B001952137801213F
:1011A800D807C00F0C1C84438B43234313701FE0E4
:1011B800DA61231C2E331B78DA0711D5631DDB7F18
:1011C800A26AFF213F2B02D85900895A89B2201CF4
:1011D80009122D300170A18D1F2B01D85B00995287
:1011E800618CA06AC9B2626B9047638F01336387D1
:1011F80038BD000010B5144C8023E0695B0082699B
:101208001A4202D00268110610D4E069802382696C
:10121800DB001A4202D0026811060ED4201CFFF728
:1012280067FF0A4B228E56331A8010BDC361238E86
:101238000133238601F0A8F8E7E7C361238E013361
:10124800238601F0A1F8E9E78403002004030020C5
:10125800064B074A1721DA615A1CD17780225200BF
:101268005A84044A9A62044A5A63704784030020E5
:101278000054004004030020F512000808B50A1CB9
:101288000349031C0868191C00F084F9002008BDF4
:10129800D003002038B5041C124B10D01868012464
:1012A8000470002100F0C0F9211C0F4801F0CAFBAE
:1012B8009020C0050421221C00F0F8FF0FE01D68F3
:1012C8009020C0050421221C00F0F0FF281C211CDE
:1012D80000F0AAF92C700448211C01F0B3FB00208F
:1012E80038BDC046D0030020002C014008B5031CBF
:1012F800082928D8081CFEF7E3FE0505260C111D51
:10130800222618005888198880B289B2FFF7B6FFDC
:101318001AE0D88880B2FFF7BDFF15E019890B4B9A
:1013280089B21868FEF738FF0DE0188A80B2FFF717
:101338002DF908E0054B1868FEF741FF03E0034B61
:101348001868FEF735FF002008BDC0466C00002075
:10135800704700207047F0B50024C4600481C48041
:10136800012087B0011C01F0ADF990278020FF050E
:101378008002012101F08EF9012501A9022603232B
:10138800381C4B7101960E718C71CD7100F034FFD1
:10139800291C381C321C802600F08EFFF6056A4690
:1013A8000F236846137055709570042701F038F8BC
:1013B80003A9301C0F804C808D80CC800C8101F0FB
:1013C8005DFC301C602101F09CFC301C391C01F0D4
:1013D8009FFC301C802101F0A5FC301C291C01F069
:1013E80016FB301C391C2A1C01F07DFC201C07B0A0
:1013F800F0BD0000064B8022191D5202CA6705493C
:1014080058310888013080B2088000201A6070477F
:1014180000E100E00403002007B580200021C0059A
:1014280001F0F5FA074B802212021A60684600F0B4
:1014380021FF90200223C0056946009300F0DCFEDE
:1014480007BDC04600E100E010B5041C8020C005BF
:10145800042101F052FC8020C00501F0F4FB80B2A9
:10146800E0806268120C93B2002B13D08020C00574
:1014780001F0E7FB61686423090C5843FEF72AFE74
:1014880080B220816168054B090C1868FEF722FEBE
:10149800E06001E02281E36010BDC046400000200A
:1014A80008B50248FFF7D0FF08BDC046C0030020BA
:1014B800024A034B08321A607047C046A04200082F
:1014C800C0030020F0B5304B0024304E047080205B
:1014D8008DB05C8001211C80000101F0E7F8301C10
:1014E80001F0DCF9684601F089FA294B6A46019354
:1014F800301C20236946538007AD1480148101F005
:1015080041FA04230127AB80301C6023291C2B805F
:101518006F80AC81EC812C826C82099401F0A2FA74
:10152800301C082101F072FB301C291C01F0DAFA8A
:10153800301C082101F072FB301C291C01F01EFB35
:10154800301C082101F076FB802303AD1B012B80A2
:101558008023DB006B808023BB40AB80301C1723CB
:10156800291CEB802C81AC8101F05CFA301C391C01
:1015780001F04DFA0D23281C2B706F70AF7000F02E
:101588004FFF0DB0F0BDC04604030020002C014001
:10159800760400000B1C017870B5002932D01A4877
:1015A800111C824200D91949194C1A481A1992B2C9
:1015B80052115200155A89B24D43174E174AAD19A8
:1015C800174E2D0C9C19A4B264115B1164005B00CA
:1015D8001B5A245A104E4C435943A4198919090C13
:1015E800240C554354434A430E48110C2D0C01F06A
:1015F80007FB240C0B48291C01F004FB0948211C9B
:1016080001F002FB70BDC04670FD000070FDFFFFD9
:1016180055550000A032000800008F027604000033
:10162800AAAAFFFF002C014038B5074D0C1C281C46
:1016380001F0E6FA281C211C01F0E4FA281C211C00
:1016480001F0E2FA38BDC046002C0140014A024BC5
:101658001A607047D4030020D003002070477047F9
:1016680010B5041C90201021C00500F01DFE0120BB
:10167800FEF714FF0C48211C01F096F80A480121D6
:1016880001F09AF80028F9D00120FEF707FF902012
:101698001021C00500F006FE0120FEF7FFFE0248FB
:1016A80001F087F810BDC0460030014010B5041C99
:1016B80090201021C00500F0F7FD0220FEF7EEFE95
:1016C8000C48211C01F06EF80A48012101F074F859
:1016D8000028F9D00820FEF7E1FE90201021C0056F
:1016E80000F0E0FD0520FEF7D9FE024801F05EF8A3
:1016F80010BDC0460030014038B5124D01242C7091
:10170800FFF7AEFF0020FFF7ABFF8022D2010240B7
:1017180011D183049B0C08D01A125A4011094A406F
:1017280091084A4051084A402240C01342400120D3
:1017380002402A7003E00448FFF792FF0023181CB8
:1017480038BDC046E80300200140000070B5144DC4
:1017580001242C70FFF784FF0221014018D1861064
:10176800B3B2002B0ED081124E40B1B20EB2361178
:1017780071408EB232B292105640B2B211B22141CB
:10178800514021400122104041400A402A7004E0A3
:10179800E7200002FFF764FF0023181C70BDC04655
:1017A800E8030020F0B5071C802087B04001012124
:1017B80000F07CFFC020C002012101AC00F06AFFEC
:1017C8000223237103230025637158480823211C31
:1017D80001932026A571E57100F00EFD5348211CE8
:1017E800019600F009FD102301930123A3714F48CE
:1017F8000223211CE37100F0FFFC4C4803212A1C42
:1018080000F05AFD494804212A1C00F055FD2A1C05
:101818004648052100F050FD9020C005102100F039
:1018280041FD9020C005311C00F03CFD9020C00512
:10183800402100F037FD012390202371C0051023BB
:10184800211C01936571A571E57100F0D5FC90200C
:10185800C005211C019600F0CFFC90204023C00554
:10186800211C019300F0C8FC201C00F04FFF3B79BD
:10187800012B03D0083BDBB2012B07D8F0231B0157
:10188800A380012323812023A38104E0E023DB003C
:10189800A3802581A68182235B00638080239B002F
:1018A8000025638122480723211C2382E5802580A7
:1018B800E58100F039FF80211D48490100F068FFEB
:1018C80001211B4800F05AFFFA204000FEF7E6FD10
:1018D80002F02AFD3B79B860012B06D1281CFFF7DE
:1018E800BFFE1448FFF708FF1CE0032B10D1642447
:1018F800013C0020E4B2FFF7D9FE002C03D0A52854
:10190800F6D1002010E0A538431E9841C0B20BE084
:10191800E7200002FFF7A4FE0748FFF7A1FE0548ED
:10192800FFF714FF054B187807B0F0BD0004004816
:1019380000300140FFFF0000F0FF0000E803002036
:10194800034B54331A88013292B21A807047C0464A
:1019580004030020F8B50379051C012B1AD1284887
:10196800FFF7CAFE274E00243378A3420BD1841117
:101978002548FFF7C1FE3378A4B2002B03D1FF231B
:1019880098432418A4B23378002B33D0FFF7D8FF3C
:101998001E4C2FE0032B2CD002F0C6FCAB68C01AFB
:1019A800F423FF339842F7D91948FFF759FE19482D
:1019B800FFF7CCFE134E071C3378002B01D0002410
:1019C800E1E71248FFF7C2FE3278002AF7D1C021BA
:1019D8008900BF00FF2280240140BA4324018A18ED
:1019E8000440141980225201031C13409B10E41870
:1019F800C9E7002402F098FCA860201CF8BDC04686
:101A0800FE7F0000E8030020FD7F0000FFFF0000CC
:101A1800F0FF0000B5E60000F8B50379061C364D66
:101A2800012B04D13548FFF767FE041C50E0032B57
:101A380034D1012300202B70FFF738FE041E102C30
:101A48001BD10020FFF732FE061C201CFFF72EFEDC
:101A5800F023334005D18000B602294A0643168098
:101A68002B700020FFF722FE264BA5283ED01A78BF
:101A7800511C1970132AF4D938E0A5280BD1214A32
:101A88001378591C1170142B03D91020FFF70EFE80
:101A980001E000232B701A4B1C8819E002F044FC6B
:101AA800B368194FC01AFA235B0098420DD913483E
:101AB800FFF74CFE33798405082B00D0040502F0AB
:101AC80033FCA40CB0603C8002E000233C882B70FF
:101AD8002B78002B03D0FFF733FF002409E00B4BD2
:101AE80058331A88013292B21A8002E000221A7022
:101AF800D1E7201CF8BDC046E8030020FFFF000026
:101B0800D6030020E9030020D803002004030020A6
:101B1800024A034B08321A607047C046C0420008A8
:101B2800DC03002008B5FEF7B9FF08BD08B502F0D0
:101B3800FBFB124B1A68811A114A91421CD9186092
:101B4800104B5A8F104B198891420ED0902080214B
:101B5800C00509011A8000F09FFB012805D19020DB
:101B68008021C0050901002204E090208021C005E1
:101B78000901012200F09AFB08BDC046EC030020D1
:101B8800400D030084030020EA03002070478623E9
:101B98009B00C3589BB2C018007D704786239B00EA
:101BA800C258C358120C9BB2D01AC0B270478523D2
:101BB8009B00C258C35892B21B0CD31AFF209843FB
:101BC800704787239B00C358DBB2C01886239B004D
:101BD800C01801234371704738B586239B00C2584B
:101BE800041C92B28218157DC268517D1F221140D3
:101BF80001228A40111C0F4AD167C158C25889B2C4
:101C0800120C914208D0C25892B2013292B2C2521A
:101C1800C258D2B2C25201E0FEF7BAFBE368281CF0
:101C28005A7D1F231A40012393401A1C024B1A6045
:101C380038BDC04604E100E000E100E010B5041C36
:101C48002368201CDB689847002802D1FEF7A0FB18
:101C580010BD2368201C5B6898473E28F6D023688F
:101C6800201C1B689847EBE738B5041C0D1C23683B
:101C7800201C1B6998470028F9D085239B00E2584F
:101C880092B2A2181132FF321571E0681F22417D0D
:101C980011400122101C8840011C0B48C167E05804
:101CA80080B2801880B2E052E058C0B2E052074BD0
:101CB800196088239B00E35C002B03D1606804490A
:101CC80001F00CF938BDC04604E100E000E100E095
:101CD8000701070030B5037A87B0013BDBB2041C6B
:101CE800042B03D8214A9B009D5801E0E1256D0291
:101CF8006068002101F0E8F8606801F01DF8002331
:101D08000293059323690095049387239B00E35866
:101D1800DBB2002B05D080235B0101938023DB001D
:101D280000E0019360686946039301F06FF8802131
:101D38006068490101F0EAF885239B00E258606871
:101D4800120CE25286239B00E258094B92B2E252EF
:101D5800084B00221A71012101F0B6F860680649A3
:101D6800012201F0BBF807B030BDC046E0420008D0
:101D78001A020000C80200200501050030B5036101
:101D8800872302729B000022C160C2540B7B85B07E
:101D9800041C0A7D0869191C00F08EFA02AD0223A2
:101DA8002B7103236B71E368291C5A891869029205
:101DB8000122AA71EA7100F01FFAE3685868002846
:101DC80001D10422226122690C2A0DD199781A7A4C
:101DD80000F072FAE368291C1A88586802920022F7
:101DE800AA71EA7100F008FAE26801A8537D03704D
:101DF800032343700123837000F012FB201CFFF7BC
:101E080069FF05B030BD000008B5064800F0E6FAE5
:101E1800032000F0E9FA012000F0ECFA00F0F0FAF3
:101E280008BDC0465555000008B500F0F1FA08BDD8
:101E3800F7B5102000F05EFB8020C002012100F001
:101E480029FC8020800301210124022600F03AFCAD
:101E580003256B461E715D719C71DC7169464023D8
:101E68004F48009300F0C8F9802369464C48009316
:101E780000F0C2F9221C4A48062100F01DFA221C73
:101E88004748072100F018FA8020211C800200F042
:101E980019FC8020211C800200F0FCFBC020211CC2
:101EA800C00200F0F7FB6B4600275D719025ED0539
:101EB8001E719F71DC718023A340281C6946009322
:101EC80000F09AF9281C80236946009300F094F9E1
:101ED8008023B340281C6946009300F08DF96946B9
:101EE8002F48009400F088F98023DB00281C6946FD
:101EF800009300F081F969462948009600F07CF9C2
:101F0800281C321C082100F0D7F9281C321C072194
:101F180000F0D2F9281C321C092100F0CDF9391C37
:101F2800321C1F4800F0C8F9281C321C0A2100F096
:101F3800C3F9321C211C1A4800F0BEF96B465F71C8
:101F48009F71281C1C7169460423009300F054F902
:101F58008020211C800200F09DFB6B461F715F7181
:101F68009F71DE71281C20236946009300F044F914
:101F78004023281C6946009300F03EF98020211C6C
:101F8800800200F087FB6B465F719F71DF711C71E7
:101F980080231B01281C6946009300F02DF9F7BD2A
:101FA80000040048024B1A8801321A807047C04664
:101FB800A402002038B59024E405201C402100F03C
:101FC80065F92021051C201C00F060F96D002843EC
:101FD800C0B238BD394B73B59A1C7921D1871A1C08
:101FE8004E320025142111805D811D8154331D80DE
:101FF800FEF790FAFFF71CFFFEF73EFAFFF704FF23
:10200800FEF704FAFFF7D6FF2D4C061C231C3833C5
:10201800E0691D7000F062F980231B0219366361C4
:10202800F6B2284BE069211C76002360E560656004
:10203800A5602661A56100F06BF9E069012100F057
:1020480099F9631CDB7F01A8037001238370457035
:1020580000F0E6F9E3691C4A596825860A405A6087
:102068001A6876218A431A601A6888210A431A6016
:10207800164B1C68201CFEF785F8154B1868FFF7EF
:1020880021FA6420FEF724FA02F04EF9051C201C00
:10209800FEF7DCF80F4A1088411C11800A21FEF770
:1020A8005DF80D4B89B219700C4B8900CB589847D5
:1020B80002F03AF9401B6328FAD9E5E70403002047
:1020C80084030020220C9410FF7FFFFF6C00002087
:1020D800D0030020A6020020A80200203832000801
:1020E8007047FEE77047704770B5074B074D0024EF
:1020F800ED1AAD101E1CAC4204D0A300F35898474B
:102108000134F8E770BDC046AC440008CC44000870
:1021180008B5074B984209D180208000012100F0C2
:10212800DDFA80208000002100F0D8FA08BDC04602
:10213800002401400B688A6810B51A43CB68C4684C
:102148001A430B691A434B691A43044B2340134340
:102158000A7952031343C36010BDC04603D2FFFF80
:102168000023036003718360C360036143617047A8
:1021780083680122002900D102221343836070473B
:10218800836A1943816242617047826880231B0613
:1021980013438360F0231B028268013BD20FD207EE
:1021A800002B01D0002AF7D18368002B01DB006CDB
:1021B80000E000207047836804221343836070475F
:1021C800006C80B270474368002A02D0194341600E
:1021D80001E08B4343607047CB0103D58268044B11
:1021E800134000E003680B40591E8B41D8B270477A
:1021F800FFFFFFFE01607047F7B50B6801930023EE
:102208000124019A9C402240A2422ED10D796C1ED5
:10221800E4B2012C15D887685C000326A640B743B2
:102228004E7987608768A640341C3C4384604468C4
:10223800A4B2944384808A7944689A40224392B233
:1022480082805A00032407689440E44327400760CB
:10225800076895403D430560C5682C40CD79C4604A
:10226800C46895402A1C2243C2600133102BC7D191
:10227800F7BD0000044B0122036000230371427183
:102288008371C3717047C046FFFF000000690840B2
:10229800431E9841C0B2704740690840431E9841A8
:1022A800C0B270478161704701857047002A01D02C
:1022B800816100E00185704707230B40C908890048
:1022C800401810B5016A9B000F249C40A14301628D
:1022D800016A9A40131C0B43036210BD08B50B4BEF
:1022E800984207D180208003012100F003FA802062
:1022F800800306E08020C003012100F0FBF9802064
:10230800C003002100F0F6F908BDC04600540040A3
:10231800026801239A43026030B5134A04688D6845
:1023280022402C0222434C680D68224302600F4A67
:10233800CC682A400261026813430360002383606B
:102348008A69C3600B6913438360826880231B0218
:10235800134383600368234303604268044B1340BC
:102368004A691343436030BDFFE0CF00FFFFFFF031
:10237800FF7FFF0701230268002901D0134301E012
:102388009A43131C03607047026801239A43026052
:1023980002680268134303607047000030B545685F
:1023A800064C89052C40039D2C4323438C0D191C96
:1023B800214314040A1C2243426030BD009800FCEB
:1023C80081627047406AC0B2704780690840431E06
:1023D8009841C0B27047C16170470000014B186056
:1023E8007047C04600300040014B58607047C046F7
:1023F80000300040014B98607047C04600300040F4
:10240800014A024B1A607047AAAA00000030004037
:10241800014A024B1A607047CCCC000000300040E3
:10242800827870B50378002A1DD09908124A0324CF
:10243800890089182340C022A3409200FF248D58A8
:10244800261C9E40B5434678B60134409C402B1C60
:1024580023438B5002781F231A40012393401A1CF0
:10246800054B1A6006E01F22134001229A40131CF4
:10247800024AD36770BDC04600E100E004E100E015
:10248800114B012219681143196058680F4901401E
:10249800596018680E490140196018680D490140D3
:1024A800196058680C4901405960D96A0F20814366
:1024B800D962186B094901401963596B914300228D
:1024C80059639A607047C046001002400CB8FFF884
:1024D800FFFFF6FEFFFFFBFFFFFFC0FFACFEF0FFB4
:1024E800034B03215A688A43104358607047C0461B
:1024F80000100240044B10211A6B8A431A631A6BAE
:10250800104318637047C04600100240F8B55A4D92
:10251800041C68680C231840FDF7D2FD1F1F1F1FFD
:102528001F1F1F1F071F1F1F1D006E68C023B60235
:102538006A68360F5B0202361A4201D14F4807E03B
:102548004D4B4F48D96A0F2319400131FDF7C2FDA1
:102558007043206004E04B4B00E0494B23600020AF
:102568006B68494A1B061B0F2168D35C0E1CDE40B2
:102578006660331C6E687605760F925DD340A36063
:102588002A6BD60501D4414A06E03B4A52685604F4
:1025980001D45A0800E09A08E2602A6B560601D472
:1025A8003B4A01E08022120222612A6BD60602D43D
:1025B800334A626100E061612F6B03222E4E17429D
:1025C80001D1A36112E0376B1740012F01D1A1613E
:1025D8000CE0376B1740022F02D18022120204E070
:1025E800366B3240032A01D1254AA261C0222F6BE3
:1025F8009202214E174201D1E36118E0376B174070
:10260800BC4680277F02BC4501D1E1610FE0376BF2
:102618001740BC468027BF02BC4502D18022120267
:1026280004E0366B1640964201D1154AE261C02299
:102638002F6B1203104E174215D0376B80231740AB
:10264800DB029F4201D121620EE0316B80231140F1
:102658001B03994202D180231B0204E0336B134011
:10266800934201D1064B23622B6B1A0602D4054B09
:10267800636200E06062F8BD0010024000093D009E
:1026880000127A00006CDC0230000020809FD50028
:1026980012800000044B5A69002902D01043586187
:1026A80001E082435A61704700100240044B9A6966
:1026B800002902D01043986101E082439A61704773
:1026C80000100240044BDA69002902D01043D86197
:1026D80001E08243DA61704700100240044BDA6877
:1026E800002902D01043D86001E08243DA607047C5
:1026F80000100240044B1A69002902D010431861E7
:1027080001E082431A617047001002400023E02272
:1027180003804380D200C380038143818381C381C6
:1027280007238280038270470388C122920110B573
:102738001A40CC890B882343CC8823430C89234334
:102748004C8923438C892343134303808288094B94
:1027580013408A88134383800B8A042203820388E8
:1027680093434A8813430380828B034B134083832C
:1027780010BDC046FFF0FFFFFFF7FFFF40230288B0
:10278800002901D0134301E09A43131C03807047CA
:102798008288034B13408380838819438180704764
:1027A800FFEFFFFF0173704781817047007BC0B264
:1027B8007047808980B2704700890840431E98415D
:1027C800C0B27047054B1A68042802D1104318603C
:1027D80002E004218A431A607047C04610E000E016
:1027E800014B58607047C04610E000E0084B0128D4
:1027F80003D11A681043186008E0023004D11A683F
:1028080001218A431A6001E000229A607047C0469D
:1028180010E000E0054B02221968002801D00A43A5
:1028280001E091430A1C1A607047C04610E000E0BE
:10283800F0B5056A0124ADB2A54305848669F3277E
:10284800B6B2056ABE4332431B011A43ADB20A232E
:102858009D432C4392B2214302830184F0BD0000C2
:10286800F0B5056A1024ADB2A543058487690A4E00
:10287800056A374016023A1C32431B0392B21A43C8
:10288800ADB2A0239D432C4309010C4392B2A4B2DC
:1028980002830484F0BDC046FF0C000008B5314B2C
:1028A800984207D1802000010121FFF717FF8020FF
:1028B800000152E08023DB05984205D10120011C6C
:1028C800FFF718FF012024E0274B984205D102208A
:1028D8000121FFF70FFF02201BE0244B984205D18E
:1028E80010200121FFF706FF102012E0204B98422C
:1028F80005D120200121FFF7FDFE202009E01D4B16
:1029080098420AD1802040000121FFF7F3FE802081
:1029180040000021FFF7EEFE22E0174B984207D156
:10292800802040020121FFF7D9FE8020400214E0F8
:10293800124B984207D1802080020121FFF7CEFE7A
:102948008020800209E00E4B984209D18020C00205
:102958000121FFF7C3FE8020C0020021FFF7BEFE61
:1029680008BDC046002C0140000400400010004093
:102978000014004000200040004001400044014095
:10298800004801400368164A30B59BB2904206D011
:102998008024E405A04202D0124CA04203D1702446
:1029A800A3434C882343104CA04203D00F4D0C89FD
:1029B8002B40234303804B68C3620B8803859042F6
:1029C80008D00B4B984205D00A4B984202D00A4BCC
:1029D800984201D18B7A03860123838230BDC04699
:1029E800002C01400004004000100040FFFCFFFFE5
:1029F80000400140004401400048014001235B427F
:102A08004360002303800381438083727047026818
:102A1800012392B2002901D0134301E09A43131C09
:102A2800038070474A880B88063013438A8813430B
:102A3800CA8813430A8913434A8913438A8913436B
:102A4800C3877047831D002904D0416C044A0A4398
:102A580092B202E0426C5204520CDA877047C046C8
:102A68000080FFFF036A01229BB29343038470B581
:102A7800056A426884697323A4B29C430B88ADB28B
:102A88001C4302239D434E888B8992B233432B43C8
:102A98000F4DA84208D00F4DA84205D00E4DA842B0
:102AA80002D00E4DA8420DD10825AB43CD894E8AE0
:102AB8002B430425AB438D882B43094D2A400D8AAF
:102AC80035432A4382808A6804834263038470BD45
:102AD800002C0140004001400044014000480140F2
:102AE800FFFCFFFF036A10229BB293430384026A30
:102AF80070B543681C4C856992B225400C889BB21E
:102B0800240225432024A2438C89ADB22401224308
:102B18004C8892B224012243144C92B2A04202D0B3
:102B2800134EB04219D1134E33400E8AB6003343C8
:102B38009BB2A04211D18024A243CC892401224314
:102B480092B24024A2438C88240122430A4C92B2B8
:102B580023404C8AA40023439BB283808B6805835F
:102B68008363028470BDC046FF8C0000002C0140C6
:102B780000400140FFFBFFFFFFF7FFFF026A1A4B0F
:102B880030B513400384056A4268C4697323A4B24C
:102B98009C430B8892B21C43144B2B408D892D0209
:102BA8002B434D889BB22D022B43114D9BB2A8425B
:102BB80014D1104D2B40CD892D022B430E4D2B40A7
:102BC8008D882D022B430D4D9BB22A400D8A2D0175
:102BD8002A434D8A92B22D012A4392B282808A6892
:102BE8008483C263038430BDFFFE0000FFFD000044
:102BF800002C0140FFF7FFFFFFFB0000FFCFFFFFA6
:102C08004163704781637047C163704783690822D5
:102C18009BB2934319430183704700008269044BB8
:102C28001A400B02111C194389B201837047C04630
:102C3800FFF70000C36908229BB2934319438183BD
:102C48007047406B7047806B704783690C229BB25A
:102C58009343038383699BB2194301837047000040
:102C68008269054B09021340038383699BB21943A8
:102C780089B201837047C046FFF30000F8B50C1C09
:102C8800A2884988051C561E20884F424F41731E52
:102C98009E4102239E1B7F002389002811D1281CF6
:102CA800FFF7C6FDE188281CFFF7CFFF281C391C59
:102CB8002389321CFFF7D4FDE188281CFFF7D0FFD9
:102CC80010E0281CFFF7CCFDE188281CFFF7C8FF9F
:102CD800281C391C2389321CFFF7AAFDE188281C0F
:102CE800FFF7B3FFF8BDC3689BB2002A02D01943AF
:102CF800818101E08B4383817047C94389B2018296
:102D08007047836870229BB29343194301817047CF
:102D1800836807229BB29343038183689BB219435C
:102D280001817047836880229BB293430381836843
:102D38009BB219430181704708B52C4B984207D1C3
:102D48008020C0010121FFF7C9FC8020C00148E0B4
:102D5800274B984207D1802080020121FFF7CAFC47
:102D6800802080021FE0234B984207D18020C002B8
:102D78000121FFF7BFFC8020C00214E01E4B9842DF
:102D880007D1802000030121FFF7B4FC8020000355
:102D980009E01A4B98420AD1802040030121FFF72D
:102DA800A9FC802040030021FFF7A4FC1CE0144B81
:102DB800984205D120200121FFF790FC202010E047
:102DC800104B984205D140200121FFF787FC402095
:102DD80007E00D4B984207D180200121FFF77EFCC8
:102DE80080200021FFF77AFC08BDC046003801406A
:102DF8000044004000480040004C004000500040A3
:102E08000014014000180140001C01400368012221
:102E18009343F0B503604268244B0D1C8968134046
:102E28000B4343600268224B69681A40EB688BB019
:102E38000B432969041C0B431343036082681D4B31
:102E480013406A69134383606846FFF75FFB1A4BB8
:102E58009C4201D1069E0AE0184B9C4201D1079E74
:102E680005E0174B9C4201D1089E00E0029E2368B2
:102E78002F68190400D57600391C301CFDF72AF993
:102E8800391C051C301CFDF769F97F080023B9427D
:102E98005B41ED1823681A0404D50A4A2B075B0F17
:102EA80015401D43ADB2A5810BB0F0BDFFCFFFFFAC
:102EB800F3E9FFFFFFFCFFFF00380140004400403A
:102EC80000480040F0FF000001230268002901D0FB
:102ED800134301E09A43131C036070478BB210B58B
:102EE800C9B201248C401B0A211C022B01D10430D9
:102EF80002E0032B00D108300368002A02D01943EE
:102F0800016001E08B43036010BD00008268034B41
:102F1800134083608368194381607047FFEFFFFFA8
:102F2800CBB210B501248AB29C40120A231C012A94
:102F380001D1026804E0022A01D1426800E08268F7
:102F48001340C2690020834208D0090C0120884040
:102F5800011C101C0840411E8841C0B210BD000071
:102F68001348854613480168090E134A914205D152
:102F7800124813490160134813490160002103E016
:102F8800124B5B58435004311148124B42189A4275
:102F9800F6D3114A02E00023136004320F4B9A4221
:102FA800F9D300F01FF8FFF79FF8FFF713F8FEE7D3
:102FB80000200020040000001F000000181002403C
:102FC800010000000000014000000000CC4400089F
:102FD800000000204400002044000020F0030020EE
:102FE800FEE70000454B13B519680122114319602B
:102FF80058684349014059601868424901401960BE
:1030080018684149014019605868404901405960B1
:10301800D96A0F208143D962186B3D490140196371
:10302800596B9143002259639A6000920192196882
:10303800802252020A431A601A68802189020A40D3
:103048000192009A01320092019A002A04D1009854
:10305800A022D2019042EFD11868284A014002D03C
:103068000122019204E0019110682A49014011608F
:1030780029491120019C08605968284A59605968F3
:10308800596059680A405A605968012C1AD1882237
:1030980052030A435A601968802282400A431A6020
:1030A8001968164A8801FBD551680320814351608D
:1030B800516802200143516059680C220A40082ACD
:1030C800FAD119E0A02292030A435A6019688022B3
:1030D80052040A431A601968084A8801FBD55168E6
:1030E80003208143516051680220014351605968AF
:1030F8000C220A40082AFAD113BDC046001002402B
:103108000CB8FFF8FFFFF6FEFFFFFBFFFFFFC0FF55
:10311800ACFEFFFFFFFFFEFF00200240FF7FC0FF65
:10312800F0B54F464646C0B483B0830752D0541E0C
:10313800002A4AD0CEB2031C032503E0621E002CED
:1031480043D0141C01335A1E16702B42F6D1032C9F
:1031580033D9FF250D402A0215432A0415430F2CA5
:103168001AD9271C103F3F09B9463F01B846102716
:10317800FF18BC4646461A1C6644156055609560A3
:10318800D5601032B242F8D14F4601373F010F22C5
:10319800DB191440032C10D9271F1E1DBF080196E8
:1031A800BE00B446019E1A1C664420C2B242FCD13D
:1031B8000137BF000322DB191440002C05D0C9B227
:1031C8001C1919700133A342FBD103B00CBC904603
:1031D8009946F0BD031C141CB9E7C0460000000066
:1031E80000000000000000007D01000881010008C7
:1031F8008301000887010008890100080000000019
:103208000000000000000000B5030008C303000828
:10321800DD030008F303000800400E00000000482A
:10322800010000800F00000000000048011C0000A1
:103238002D1B0008351B0008951B00081105000808
:1032480013050008150500081705000819050008EA
:103258001B050008AD1F000800000000000000006A
:10326800AD0500085506000889060008AB050008EA
:10327800A705000800000000000000000000000092
:10328800B50E00082D0E00087D0F00082B0E000853
:10329800310E000800000000FF7F6480C8802D8187
:1032A8009181F6815A82BF8223838883EC8351847B
:1032B800B5841A857E85E2854786AB861087748734
:1032C800D8873D88A18805896989CE89328A968AF6
:1032D800FA8A5E8BC38B278C8B8CEF8C538DB78DC2
:1032E8001B8E7F8EE28E468FAA8F0E907190D5909E
:1032F80039919C9100926392C7922A938E93F1938D
:103308005494B8941B957E95E1954496A7960A9790
:103318006D97CF9732989598F8985A99BD991F9AB2
:10332800819AE49A469BA89B0A9C6C9CCE9C309DF3
:10333800929DF49D569EB79E199F7A9FDC9F3DA053
:103348009EA0FFA060A1C1A122A283A2E4A245A3DE
:10335800A5A306A466A4C7A427A587A5E7A547A68D
:10336800A7A607A766A7C6A725A885A8E4A843A96E
:10337800A2A901AA60AABFAA1EAB7CABDBAB39AC81
:1033880098ACF6AC54ADB2AD10AE6DAECBAE29AFC5
:1033980086AFE3AF40B09DB0FAB057B1B4B110B248
:1033A8006DB2C9B225B382B3DEB339B495B4F1B402
:1033B8004CB5A7B503B65EB6B9B614B76EB7C9B7FC
:1033C80023B87DB8D8B832B98BB9E5B93FBA98BA3D
:1033D800F1BA4BBBA4BBFDBB55BCAEBC06BD5FBDC3
:1033E800B7BD0FBE67BEBEBE16BF6DBFC4BF1CC093
:1033F80072C0C9C020C176C1CDC123C279C2CFC2B3
:1034080024C37AC3CFC324C479C4CEC423C577C523
:10341800CCC520C674C6C8C61BC76FC7C2C715C8E7
:1034280068C8BBC80EC960C9B3C905CA57CAA8CA03
:10343800FACA4BCB9CCBEDCB3ECC8FCCDFCC30CD7E
:1034480080CDD0CD1FCE6FCEBECE0DCF5CCFABCF53
:10345800FACF48D096D0E4D032D180D1CDD11AD28B
:1034680067D2B4D201D34DD39AD3E6D331D47DD425
:10347800C8D414D55FD5A9D5F4D53ED689D6D2D629
:103488001CD766D7AFD7F8D741D88AD8D2D81BD996
:1034980063D9ABD9F2D93ADA81DAC8DA0EDB55DB6F
:1034A8009BDBE1DB27DC6DDCB2DCF8DC3DDD81DDBC
:1034B800C6DD0ADE4EDE92DED6DE19DF5CDF9FDF78
:1034C800E2DF24E067E0A9E0EAE02CE16DE1AEE1AB
:1034D800EFE130E270E2B0E2F0E230E36FE3AEE356
:1034E800EDE32CE46BE4A9E4E7E424E562E59FE579
:1034F800DCE519E655E692E6CEE609E745E780E71A
:10350800BBE7F6E731E86BE8A5E8DFE818E951E939
:103518008AE9C3E9FCE934EA6CEAA3EADBEA12EBDC
:1035280049EB80EBB6EBECEB22EC58EC8DECC2EC03
:10353800F7EC2CED60ED94EDC8EDFCED2FEE62EEAE
:1035480095EEC7EEFAEE2BEF5DEF8FEFC0EFF1EFE0
:1035580021F052F082F0B1F0E1F010F13FF16EF19C
:103568009CF1CAF1F8F126F253F280F2ADF2DAF2E8
:1035780006F332F35DF389F3B4F3DFF309F434F4BB
:103588005EF487F4B1F4DAF403F52CF554F57CF520
:10359800A4F5CBF5F2F519F640F666F68CF6B2F618
:1035A800D7F6FDF621F746F76AF78EF7B2F7D6F7A2
:1035B800F9F71CF83EF861F883F8A4F8C6F8E7F8BC
:1035C80008F928F949F969F988F9A8F9C7F9E5F96D
:1035D80004FA22FA40FA5EFA7BFA98FAB5FAD1FAB6
:1035E800EDFA09FB25FB40FB5BFB76FB90FBAAFB96
:1035F800C4FBDDFBF7FB0FFC28FC40FC58FC70FC0F
:1036080087FC9EFCB5FCCCFCE2FCF8FC0DFD23FD20
:1036180038FD4CFD61FD75FD88FD9CFDAFFDC2FDCB
:10362800D4FDE7FDF9FD0AFE1CFE2DFE3DFE4EFE13
:103638005EFE6EFE7DFE8CFE9BFEAAFEB8FEC6FEFA
:10364800D4FEE1FEEEFEFBFE08FF14FF20FF2BFF79
:1036580036FF41FF4CFF56FF60FF6AFF73FF7CFF98
:1036680085FF8EFF96FF9EFFA5FFACFFB3FFBAFF55
:10367800C0FFC6FFCCFFD1FFD7FFDBFFE0FFE4FFB1
:10368800E8FFEBFFEFFFF2FFF4FFF6FFF8FFFAFFAA
:10369800FCFFFDFFFDFFFEFFFEFFFEFFFDFFFDFF40
:1036A800FCFFFAFFF8FFF6FFF4FFF2FFEFFFEBFF76
:1036B800E8FFE4FFE0FFDBFFD7FFD1FFCCFFC6FF49
:1036C800C0FFBAFFB3FFACFFA5FF9EFF96FF8EFFBA
:1036D80085FF7CFF73FF6AFF60FF56FF4CFF41FFC9
:1036E80036FF2BFF20FF14FF08FFFBFEEEFEE1FE76
:1036F800D4FEC6FEB8FEAAFE9BFE8CFE7DFE6EFEC4
:103708005EFE4EFE3DFE2DFE1CFE0AFEF9FDE7FDA7
:10371800D4FDC2FDAFFD9CFD88FD75FD61FD4CFD2E
:1037280038FD23FD0DFDF8FCE2FCCCFCB5FC9EFC4D
:1037380087FC70FC58FC40FC28FC0FFCF7FBDDFB09
:10374800C4FBAAFB90FB76FB5BFB40FB25FB09FB5C
:10375800EDFAD1FAB5FA98FA7BFA5EFA40FA22FA4B
:1037680004FAE5F9C7F9A8F988F969F949F928F9CE
:1037780008F9E7F8C6F8A4F883F861F83EF81CF8E9
:10378800F9F7D6F7B2F78EF76AF746F721F7FDF69D
:10379800D7F6B2F68CF666F640F619F6F2F5CBF5E2
:1037A800A4F57CF554F52CF503F5DAF4B1F487F4B7
:1037B8005EF434F409F4DFF3B4F389F35DF332F320
:1037C80006F3DAF2ADF280F253F226F2F8F1CAF11A
:1037D8009CF16EF13FF110F1E1F0B1F082F052F09E
:1037E80021F0F1EFC0EF8FEF5DEF2BEFFAEEC7EEB0
:1037F80095EE62EE2FEEFCEDC8ED94ED60ED2CED4C
:10380800F7ECC2EC8DEC58EC22ECECEBB6EB80EB71
:1038180049EB12EBDBEAA3EA6CEA34EAFCE9C3E918
:103828008AE951E918E9DFE8A5E86BE831E8F6E745
:10383800BBE780E745E709E7CEE692E655E619E6F5
:10384800DCE59FE562E524E5E7E4A9E46BE42CE424
:10385800EDE3AEE36FE330E3F0E2B0E270E230E2D2
:10386800EFE1AEE16DE12CE1EAE0A9E067E024E0F8
:10387800E2DF9FDF5CDF19DFD6DE92DE4EDE0ADE96
:10388800C6DD81DD3DDDF8DCB2DC6DDC27DCE1DBAB
:103898009BDB55DB0EDBC8DA81DA3ADAF2D9ABD931
:1038A80063D91BD9D2D88AD841D8F8D7AFD766D729
:1038B8001CD7D2D689D63ED6F4D5A9D55FD514D58E
:1038C800C8D47DD431D4E6D39AD34DD301D3B4D25E
:1038D80067D21AD2CDD180D132D1E4D096D048D097
:1038E800FACFABCF5CCF0DCFBECE6FCE1FCED0CD33
:1038F80080CD30CDDFCC8FCC3ECCEDCB9CCB4BCB31
:10390800FACAA8CA57CA05CAB3C960C90EC9BBC88A
:1039180068C815C8C2C76FC71BC7C8C674C620C643
:10392800CCC577C523C5CEC479C424C4CFC37AC354
:1039380024C3CFC279C223C2CDC176C120C1C9C0B8
:1039480072C01CC0C4BF6DBF16BFBEBE67BE0FBE6F
:10395800B7BD5FBD06BDAEBC55BCFDBBA4BB4BBB74
:10396800F1BA98BA3FBAE5B98BB932B9D8B87DB8C7
:1039780023B8C9B76EB714B7B9B65EB603B6A7B55C
:103988004CB5F1B495B439B4DEB382B325B3C9B23A
:103998006DB210B2B4B157B1FAB09DB040B0E3AF58
:1039A80086AF29AFCBAE6DAE10AEB2AD54ADF6ACAE
:1039B80098AC39ACDBAB7CAB1EABBFAA60AA01AA42
:1039C800A2A943A9E4A885A825A8C6A766A707A70A
:1039D800A7A647A6E7A587A527A5C7A466A406A402
:1039E800A5A345A3E4A283A222A2C1A160A1FFA02E
:1039F8009EA03DA0DC9F7A9F199FB79E569EF49D7E
:103A0800929D309DCE9C6C9C0A9CA89B469BE49AF8
:103A1800819A1F9ABD995A99F89895983298CF9794
:103A28006D970A97A7964496E1957E951B95B8944D
:103A38005494F1938E932A93C792639200929C9127
:103A48003991D59071900E90AA8F468FE28E7F8E15
:103A58001B8EB78D538DEF8C8B8C278CC38B5E8B15
:103A6800FA8A968A328ACE8969890589A1883D8829
:103A7800D88774871087AB864786E2857E851A8546
:103A8800B5845184EC8388832383BF825A82F6816C
:103A980091812D81C8806480FF7F9A7F367FD17E97
:103AA8006D7E087EA47D3F7DDB7C767C127CAD7BC1
:103AB800497BE47A807A1C7AB7795379EE788A78E8
:103AC8002678C1775D77F97695763076CC75687506
:103AD8000475A0743B74D77373730F73AB7247721A
:103AE800E3717F711C71B8705470F06F8D6F296F1E
:103AF800C56E626EFE6D9B6D376DD46C706C0D6C0F
:103B0800AA6B466BE36A806A1D6ABA695769F468EA
:103B180091682F68CC6769670667A4664166DF65A8
:103B28007D651A65B8645664F46392633063CE6247
:103B38006C620A62A8614761E56084602260C15FC7
:103B4800605FFF5E9E5E3D5EDC5D7B5D1A5DB95C1D
:103B5800595CF85B985B375BD75A775A175AB7594D
:103B68005759F75898583858D95779571A57BB564C
:103B78005C56FD559E553F55E05482542354C55319
:103B880066530853AA524C52EE5191513351D550B5
:103B980078501B50BE4F614F044FA74E4A4EEE4D12
:103BA800914D354DD94C7C4C204CC54B694B0D4B38
:103BB800B24A574AFB49A0494549EA48904835481E
:103BC800DB4781472647CC4673461946BF456645BD
:103BD8000D45B3445A440144A9435043F8429F4217
:103BE8004742EF4197414041E84091403A40E23F27
:103BF8008C3F353FDE3E883E313EDB3D853D2F3DE7
:103C0800DA3C843C2F3CDA3B853B303BDB3A873A55
:103C1800323ADE398A393639E3388F383C38E93771
:103C280096374337F0369E364B36F935A735563535
:103C38000435B33462341134C0336F331F33CE329A
:103C48007E322E32DF318F314031F130A2305330A5
:103C58000430B62F682F1A2FCC2E7E2E312EE42D4D
:103C6800972D4A2DFD2CB12C642C182CCD2B812B93
:103C7800362BEA2A9F2A552A0A2AC02975292C296F
:103C8800E22898284F280628BD2774272C27E326E2
:103C98009B2653260C26C4257D253625F024A924E9
:103CA80063241D24D72391234C230623C1227D227C
:103CB8003822F421B0216C212821E520A2205F20A0
:103CC8001C20DA1F971F551F141FD21E911E501E4D
:103CD8000F1ECE1D8E1D4E1D0E1DCE1C8F1C501C82
:103CE800111CD21B931B551B171BDA1A9C1A5F1A3F
:103CF800221AE519A9196C193019F518B9187E187E
:103D080043180818CD17931759171F17E616AD163D
:103D180074163B160216CA1592155B152315EC147A
:103D2800B5147E1448141214DC13A61371133C1333
:103D38000713D2129E126A1236120212CF119C1168
:103D4800691137110411D310A1106F103E100D1016
:103D5800DD0FAC0F7C0F4D0F1D0FEE0EBF0E900E3A
:103D6800620E340E060ED80DAB0D7E0D510D240DCE
:103D7800F80CCC0CA10C750C4A0C1F0CF50BCA0BDB
:103D8800A00B770B4D0B240BFB0AD20AAA0A820A56
:103D98005A0A330A0C0AE509BE09980972094C093E
:103DA80027090109DD08B808940870084C08280894
:103DB8000508E207C0079D077B075A07380717075A
:103DC800F606D606B5069506760656063706190689
:103DD800FA05DC05BE05A0058305660549052D0520
:103DE8001105F504D904BE04A30488046E04540420
:103DF8003A0421040704EF03D603BE03A6038E0387
:103E080077036003490332031C030603F102DB0254
:103E1800C602B2029D028902760262024F023C0289
:103E28002A0217020502F401E201D101C101B00121
:103E3800A00190018101720163015401460138011A
:103E48002A011D0110010301F600EA00DE00D3007B
:103E5800C800BD00B200A8009E0094008B0082003C
:103E68007900700068006000590052004B0044005F
:103E78003E00380032002D00270023001E001A00E3
:103E8800160013000F000C000A00080006000400CA
:103E98000200010001000000000000000100010014
:103EA80002000400060008000A000C000F001300BE
:103EB80016001A001E00230027002D0032003800CB
:103EC8003E0044004B00520059006000680070003A
:103ED800790082008B0094009E00A800B200BD000B
:103EE800C800D300DE00EA00F600030110011D013E
:103EF8002A013801460154016301720181019001D0
:103F0800A001B001C101D101E201F40105021702CB
:103F18002A023C024F026202760289029D02B20224
:103F2800C602DB02F10206031C03320349036003E5
:103F380077038E03A603BE03D603EF030704210409
:103F48003A0454046E048804A304BE04D904F50496
:103F580011052D05490566058305A005BE05DC0587
:103F6800FA0519063706560676069506B506D606E4
:103F7800F606170738075A077B079D07C007E207A9
:103F8800050828084C0870089408B808DD080109D5
:103F980027094C0972099809BE09E5090C0A330A70
:103FA8005A0A820AAA0AD20AFB0A240B4D0B770B7B
:103FB800A00BCA0BF50B1F0C4A0C750CA10CCC0CF2
:103FC800F80C240D510D7E0DAB0DD80D060E340ED8
:103FD800620E900EBF0EEE0E1D0F4D0F7C0FAC0F34
:103FE800DD0F0D103E106F10A110D3100411371102
:103FF80069119C11CF11021236126A129E12D21246
:1040080007133C137113A613DC13121448147E14FF
:10401800B514EC1423155B159215CA1502163B1638
:104028007416AD16E6161F1759179317CD170818EB
:1040380043187E18B918F51830196C19A919E5191B
:10404800221A5F1A9C1ADA1A171B551B931BD21BCC
:10405800111C501C8F1CCE1C0E1D4E1D8E1DCE1DFE
:104068000F1E501E911ED21E141F551F971FDA1FB8
:104078001C205F20A220E52028216C21B021F421FA
:1040880038227D22C12206234C239123D7231D24C5
:104098006324A924F02436257D25C4250C2653261F
:1040A8009B26E3262C277427BD2706284F28982807
:1040B800E2282C297529C0290A2A552A9F2AEA2A82
:1040C800362B812BCD2B182C642CB12CFD2C4A2D92
:1040D800972DE42D312E7E2ECC2E1A2F682FB62F39
:1040E80004305330A230F13040318F31DF312E327D
:1040F8007E32CE321F336F33C03311346234B3345F
:1041080004355635A735F9354B369E36F0364337E4
:104118009637E9373C388F38E33836398A39DE390B
:10412800323A873ADB3A303B853BDA3B2F3C843CDA
:10413800DA3C2F3D853DDB3D313E883EDE3E353F56
:104148008C3FE23F3A409140E84040419741EF417F
:1041580047429F42F8425043A94301445A44B3445A
:104168000D456645BF4519467346CC4626478147E7
:10417800DB4735489048EA484549A049FB49574A32
:10418800B24A0D4B694BC54B204C7C4CD94C354D34
:10419800914DEE4D4A4EA74E044F614FBE4F1B50F6
:1041A8007850D55033519151EE514C52AA52085380
:1041B8006653C55323548254E0543F559E55FD55CC
:1041C8005C56BB561A577957D95738589858F758E4
:1041D8005759B759175A775AD75A375B985BF85BCC
:1041E800595CB95C1A5D7B5DDC5D3D5E9E5EFF5E81
:1041F800605FC15F22608460E5604761A8610A6210
:104208006C62CE6230639263F4635664B8641A6574
:104218007D65DF654166A46606676967CC672F68B8
:104228009168F4685769BA691D6A806AE36A466BDF
:10423800AA6B0D6C706CD46C376D9B6DFE6D626EE5
:10424800C56E296F8D6FF06F5470B8701C717F71D7
:10425800E3714772AB720F737373D7733B74A074B7
:1042680004756875CC7530769576F9765D77C17783
:1042780026788A78EE785379B7791C7A807AE47A46
:10428800497BAD7B127C767CDB7C3F7DA47D087E00
:104298006D7ED17E367F9A7F00000000000000000E
:1042A8005F13000821140008FD13000859130008C3
:1042B8005B13000800000000000000000000000080
:1042C800AD17000867160008211A000865160008CF
:1042D8005D1900080000000000E1000000960000E1
:1042E800004B00008025000000E8030000000000EB
:1042F8000000000000000000E11B0008971B0008F8
:10430800711C0008A51B0008B71B0008451C000805
:08431800CB1B000800000000AF
:1043200008B5024800F046F808BDC04674000020F9
:10433000094B0A49986810B5094A0C689B685443B0
:104340000968984202D8141C4C43181C0621FBF73C
:10435000C5FE201A10BDC04610E000E02800002075
:1043600040420F00044B1A6801321A60034B1A686E
:1043700001321A607047C04628000020A0020020C9
:1043800008B50948FDF720FF084B09499A898A4278
:1043900004D001329A819A688018986002480421FA
:1043A000FDF72CFF08BDC04600240140AC020020F0
:1043B000FFFF000038B53749041C4068FEF7B4FD24
:1043C000002837D06268344B506AD16980B28D07BB
:1043D00010D18622920099589D58090C0131C9B21A
:1043E000ADB2A94222D09A58120C9A1810752B4AD5
:1043F00099521FE0D26987218900D00703D45A5807
:10440000D2B2002A12D159588620C9B25918800058
:104410000918497987229200002907D1995801206B
:10442000C9B24140181C9954FDF758FC1C4B1A881E
:1044300001321A8060681B49FEF776FD002827D0FC
:10444000154B852292009858995880B2090C8842E1
:1044500011D099586568090C59181131FF31097943
:10446000298598581049000C013080B258529A584A
:10447000120CD2B25A528522920099589B58090CBC
:104480009BB2994204D1606806490022FEF72AFDDA
:1044900038BDC04605010500740000201A02000066
:0C44A00070000020070107001602000059
:1044AC004903000869040008D9060008F50F000844
:1044BC0059120008B914000855160008191B0008F9
:1044CC004800002000000000000000000000000078
:1044DC0000000000000000000000000000000000D0
:1044EC000000000000000000010000001027000088
:1044FC00000000000102030401020304060708097E
:04450C00006CDC0261
:0400000508002F6957
:00000001FF
